:1000000000100020D5470000CD430000850500000A
:1000100000000000000000000000000000000000E0
:10002000000000000000000000000000CF430000BE
:100030000000000000000000D14300006D490000F6
:10004000412900004D2900005929000065290000C0
:10005000D343000071290000474600007D290000BD
:100060008929000095290000A1290000AD29000080
:10007000B9290000C5290000D1290000DD290000B0
:10008000E9290000F5290000012A0000D5430000FD
:10009000D54300000D2A0000192A0000252A00007F
:1000A000312A00003D2A0000492A0000552A00009C
:1000B00001000000000000000A0000000000000035
:1000C0006400000000000000E803000000000000E1
:1000D0001027000000000000A086010000000000C2
:1000E00040420F00000000008096980000000000D1
:1000F00000E1F5050000000000CA9A3B0000000086
:1001000000E40B540200000000E8764817000000ED
:100110000010A5D4E800000000A0724E18090000ED
:1001200000407A10F35A00000080C6A47E8D0300C0
:100130000000C16FF286230000008A5D78456301EC
:10014000000064A7B3B6E00D0000E8890423C78A65
:1001500001238B400449C0010818002A01D08360A4
:0C016000704743607047C0460028004014
:10016C00022A0CD0012A11D0002A1BD1C001401840
:10017C000D4940184021425CFB23134011E0012241
:10018C008A40C001084BC018426105E001228A4038
:10019C00C001054BC018826140184021425C042309
:0C01AC00134343547047C0460028004035
:1001B80030B581B0C00140180749435C6C462370D4
:1001C800521E55425541AA01BF251D40AA1822704A
:0C01D800009A425401B030BD40280040A5
:1001E40030B581B0C00140180749435C6C462370A8
:1001F400551EAA415200FD251D40AA182270009ADE
:0C020400425401B030BDC046402800400C
:1002100001238B400549C0010818002A02D0416A19
:10022000194301E0416A9943416270470028004048
:1002300030B581B0C00140180649435C6C4623705C
:10024000551EAA41FE251D40AA182270009A42544C
:0802500001B030BD4028004060
:10025800F0B581B04B08C001C0180A4BC45C6D46AC
:100268002C7001270F260F4001D0120100E0324008
:10027800002F00D1F643344014432C700099C15428
:0802880001B0F0BD3028004078
:1002900001238B400449C0010818002A01D0836162
:0C02A000704743617047C04600280040D2
:1002AC0001228A40C0010149425070471C2800407D
:1002BC00C001034A8258CA40012010407047C04612
:0402CC0020280040A6
:1002D00030B581B0840014482418E56900954D1E9E
:1002E000A94109020F25154049191A048918049AD1
:1002F000531E9A4152038918059A531E9A411203BC
:100300008918069A531E9A41D2028918079A531ED9
:100310009A4192020A4300920099E1610168002922
:0C032000FCD101B030BDC0460418004004
:10032C00531E9A4192010F230B40D1188000014AB1
:08033C00815070478018004059
:1003440030B581B0441E0546A5416C008907090FEC
:100354000919541EA241920189185A1E9341DA01C7
:1003640089186A4611700549009A0A72002802D059
:100374000868C006FCD501B030BDC0460C0C004076
:1003840030B581B0441E0546A5416C004D1EA941FF
:1003940089000919541EA241920189185A1E9341D9
:1003A400DA018918049A5207520D8918059A531EC6
:1003B4009A41D2028918069A12030A4369460A80AE
:1003C4000449009A8A80002802D00868C007FCD03B
:0803D40001B030BD0C0C00402B
:1003DC0010B581B0441EA04140004C1EA1418901C2
:1003EC000818511E8A41D1014018591E4A424A41EF
:1003FC009100401869460880034800998181016882
:0C040C00C905FCD501B010BD0C0C00406F
:1004180081B0074A0A40800280B2801800900548DF
:10042800009901610168C905FCD501B07047C04653
:08043800FF0300000C0C004062
:10044000024B187059709A707047C04604040040FF
:1004500081B0421E9041C00103220A4080186946C3
:10046000087002480099017001B070470200004016
:1004700081B01148007869460870C1070ED1810724
:100480000ED441070ED4C1060ED481060ED4410607
:100490000ED40006C117062008400AE0002008E03C
:1004A000012006E0022004E0032002E0042000E036
:0C04B000052001B07047C0460008004065
:1004BC0081B00749096800910A0D82808AB20260F6
:1004CC00C90B0E220A400349895AC18001B07047FA
:0804DC0008400041C447000084
:1004E40010B581B0421E9041800407221204064BCD
:1004F4001C680094944300198907890B40180090E4
:0C0504000098186001B010BD04400041D8
:1005100081B006490A6800921E239A430007C00E64
:10052000101800900098086001B070470440004126
:1005300081B003210902064A136800938B438007A8
:10054000800D181800900098106001B07047C046E8
:040550000440004122
:1005540081B00A49096841710A0F02700A05120F35
:1005640002710A04120FC2708A02920E82700A018A
:10057400D20E4270009101B07047C046182000416D
:100584000A490A68002AFED404207146084202D1AE
:10059400EFF3088001E0EFF309800123DB071A433E
:1005A4000A60816902318161704700002CED00E02E
:1005B400034C2068241D8047FBE701F0DDFFFEE7C4
:0405C400AC51000036
:1005C800C278032313400279407900028018104A48
:1005D80002400020032B0ED0022B05D0012B16D190
:1005E80002290C490FD00FE0022908D10121490244
:1005F8008A420BD07047022904D0402104E0412AE6
:1006080004D370470349491C914200D30120704725
:08061800FF070000FF030000D2
:1006200002484078411E88417047C046C0070020FC
:10063000024800780421014088087047C007002064
:0C064000014800787047C04644090020C3
:10064C00F0B583B0024621480178012000293BD146
:10065C00019202901E48332102F02CFE1D4C201DED
:10066C0003F09AFF1C4804601C4F002F04D01C4858
:10067C0000BF00BF1B490860194E317800201A4C8E
:10068C000546002F2A4609D0EAB28A4205D2182123
:10069C00414314480068401804E06A1AD0B218218B
:1006AC0041436018006880476D1CE8B231788A1CA1
:1006BC008242E6D8019C204600F022FE204600F043
:1006CC0061FE02980149087003B0F0BD4409002096
:1006DC00C00700206009002018080020000000005E
:0C06EC00450900201C08002080100000C0
:1006F800F0B591B004F070F8002800D146E30DA8D9
:10070800001D0890AB4EAC4FAC4D346838780128CA
:1007180002D1002000F03EFE201D0DA903F0B5FE19
:1007280004463878012802D1002000F02DFE002C64
:1007380000D12BE30DA84078401E0728E5D8C04615
:100748007844007940008744030A1438444D88AE41
:100758000DA8007804F056F80E98A870D5E70DA8F3
:10076800007804F04FF8EA480028CED001F0BEFF28
:10077800CBE7E848007800210C46E74A002A2246E1
:1007880008D0E2B2824204D218224A43E3490968F7
:1007980004E0221AD1B218224A43E149891849696A
:1007A800002904D00DA800788847DA480078641C2E
:1007B800E1B2821C8A42E0D8A7E72878C107A4D012
:1007C800D8490029A1D008210840C00801F096FFA7
:1007D8009BE72878C00798D0D348002895D001F027
:1007E80095FF92E72878012109910843287023246E
:1007F800285DFE2318402855285DFB210840285510
:100808002846233042780B931A40427042780A40B7
:1008180042703D4637460DAE30780C9000200A9065
:1008280000F0E8FC31793E462F46B04D4806800F6F
:10083800032800D1AAE002283CD1BC48002800D1F6
:10084800A4E0BA4800F0D6FC00210C98089A00BF32
:1008580000BF002800D058E798E00DA801797F2054
:1008680008404200AA18CB09D2182323D45CFE25DD
:100878002540D554D45CFB252540D554002800D10B
:100888007DE2D07CA44A002A39D0A24A127890424C
:10089800964D36D2A14A1268002A00D176E2182372
:1008A8004343D31836E00E99002900D12DE70F985D
:1008B80088472AE71F220A40022A32D0012A4BD051
:1008C800002A63D16020014020294BD10DA800895E
:1008D8000106090F5AD1C0B22818C0788E490029DC
:1008E80000D1EBE18B490978884200D3E5E18B49D7
:1008F800096800294AD0182242438918E6E17B4D4D
:1009080000E0801AC0B2012800D93FE21822424311
:10091800834883180DA8427900781C690F9BA0476B
:10092800F3E60DA909897F220A40072A2ED852002A
:10093800AA18C9B20B91CB09D118CB7C764A002AE8
:1009480052D0744D2D78AB424CD20A9118255D4394
:10095800724A136859194FE00DA800890106090F5A
:100968002ED013E00DA8407909280FD84000C046C2
:10097800784480884000874413008D000900960061
:100988000900A000AD000900E100EA000DAC2078E4
:10099800002100F0E7FD2078802100F0E3FDB4E6B7
:1009A80028788108022319408006C00F401810AA31
:1009B8001080C7E01808002060090020C007002048
:1009C800C0B22818C078F349002930D0F049097816
:1009D80088422BD2F14909680029D7D0182242430E
:1009E80089182BE05B1BEE4DDBB2012B0AD80A916C
:1009F80018255D43E84A51190028E94D06D0002919
:100A0800C4D063E10028C1D10A9100210DA8407922
:100A1800032831D001282FD000280A98B6D1005DCC
:100A28008007C00F10AA108002238BE0401AC0B2C2
:100A38000128ABD818214143D74841180C98089A87
:100A480003F008FD002800D05FE60DA800794006F5
:100A5800800F9BD10DA840790B9908400A2895D1A1
:100A68000024204600F0C6FB0DA840790A2800D0D3
:100A780080E110AA147064E00DAAD288002A00D080
:100A88002EE10C46012800D025E10C980B9900F0C6
:100A9800A1FA24E10DA8C088012800D076E72878BB
:100AA800F721014007E00DA8C088012800D06DE7B4
:100AB80028780821014329705CE1089800F0A0FB20
:100AC8000DA881790C9800F06FFC28780221014369
:100AD80029701AE60DA8C088010A491E0E2900D9F6
:100AE80054E703A24900515A49008F44C007002027
:100AF800220008010C012100210012011E01210021
:100B08002100210021002100210021002901C046E7
:100B1800F526000045090020000000001C08002000
:100B280080100000052700001527000000000000C5
:100B38002CE700F061FF024612230FE1687810AA43
:100B4800107001230C98089900F0DCFADDE568784C
:100B58000DA9CC88E1B2884200D10AE16878002862
:100B680002940BD00C9C204603F081FCA8780B90D3
:100B78002046029C00F048FA0B98A870200600D185
:100B8800F7E0601EC0B200F03FFF002800D1FDE68C
:100B98004178022900D0F9E62978CF220A40C179A4
:100BA800490810230B40D21820230B40D118297074
:100BB8008178C278120251184118039109300399BB
:100BC800884200D3CFE041780B2906D1017841183B
:100BD8000B914978C078049002E0099A04920B902E
:100BE800042900D0D2E603980B99401A80B20790E6
:100BF800674800780A9C22466649002921460692E1
:100C080009D0E1B2814205D21820504363490968EE
:100C1800081809E0211AC8B2012804D8182141434C
:100C28005D48401800E00020059083680C980B99F7
:100C3800079D2A469847092802D30346854209D2C8
:100C480053480078811C641CE2B29142544DD3D8B9
:100C58000B982FE0049800281CD0012808D105988B
:100C680080685449884201D0012000E002200490A5
:100C780000200B9989780918C9B2494D6918CA78B2
:100C8800FF2A00D082E6C91C0C70401CC1B2049A2D
:100C98009142EED3424D284613301A460193E3B2EF
:100CA8000B9C214603F09CFD0198201838490978CF
:100CB800891C069A914282D868E6401AC0B2012877
:100CC80000D963E618214143334841180C98089A23
:100CD80003F0C0FBBDE50C980B9900F061F92146C3
:100CE800002900D111E50C98089A03F0B3FB002005
:100CF80000F080FA2420285CC0073BD005E5C0B28C
:100D080000F082FE18E00DA90989C0B200F080FE4B
:100D180005E02548002800D138E600BF00BF0028BC
:100D280000D133E60246037818E01E49002900D1B5
:100D38002CE6C0B200BF00BF024600280AD125E653
:100D48001A48002800D121E600BF00BF002800D1C2
:100D58001CE602469078D17809020B180C9808997D
:100D680000F0D0F975E512480028029C01D001F086
:100D7800B5FC6C700C98089900F096F9C5E40DA8BC
:100D8800427900780F9B00F05FFABDE411B0F0BD26
:100D98004509002000000000801000001C08002009
:100DA800C007002000000000000000000000000054
:080DB800E52600002D1C0000DF
:100DC00070B584B004464078801E03282BD8C046F6
:100DD0007844007940008744013C0D153048027882
:100DE000FE23134003700278FD231340037000229A
:100DF00042700BE02A480278D2072ED002780423F2
:100E0000134306E026480278D20726D00278FB2357
:100E10001340037023480568002908D0281D214687
:100E200003F092FB19E000291E480568F6D11E4E1A
:100E30003078012802D1002000F0B0FA281D2146A8
:100E400003F082FB3078012807D1002000F0A0FADF
:100E500003E013480278520701D404B070BD027851
:100E6000FB231340037001A8052242702278027010
:100E70000020039002900B480468002902D0201D36
:100E800001A9CDE7084D2878012802D1002000F003
:100E900085FA201D01A903F057FB2878D3E7C04647
:0C0EA000C0070020180800206009002096
:100EAC0070B5064688784006000F002500280CD146
:100EBC000C46074881782046FFF780FB002804D0B9
:100ECC003046214600F0FCFA0546284670BDC04667
:040EDC00C00700202B
:100EE0004806000E094A1018C909411823200A5C57
:100EF0000020D20708D123310A78520704D4087899
:100F0000042202430A7001207047C046C007002037
:100F10004806000E094A1018C909411823200A5C26
:100F20000020D20708D123310A78520704D5087867
:100F3000FB2202400A7001207047C046C007002013
:100F4000F0B581B04C06240E0F4D2C19CD09651952
:100F500023242C5DE4070026002C10D123352F78A4
:100F6000012427432F7000F031FA002808D1287897
:100F7000FE21014029702878FB2101402970344668
:0C0F8000204601B0F0BDC046C0070020B4
:100F8C004806000E044A1018C90940182321415C78
:0C0F9C00012008407047C046C00700203C
:100FA80010B54A06120E0A4B9A18CB09D4182322F8
:100FB800A25C92070AD4233400F0D4FA20780221E4
:100FC80001432170207801210143217010BDC046E2
:040FD800C00700202E
:100FDC0010B54A06120E0A4B9A18CB09D4182322C4
:100FEC00A25C92070AD5233400F0C8FA2078FD21C0
:100FFC00014021702078FE210140217010BDC046B7
:04100C00C0070020F9
:10101000F0B581B00446154D29780020144E0746DE
:10102000002E3A4608D0FAB28A4204D2182141432F
:101030001148006804E07A1AD0B2182141430D48E3
:1010400040184168204688477F1CF8B229788A1CDE
:101050008242E5D8094C3321204602F031F9E01CE8
:101060002021FF2202F02DF901B0F0BD450900203A
:1010700000000000801000001C080020C0070020B5
:10108000B11B0000051C00002D1C0000CD1C000041
:10109000B51D000000000000791F0000891F00003E
:1010A000991F0000292000002922000000000000F4
:1010B000F0B585B0049088790390C87902900879DA
:1010C00001904F798E78CC780B7848780E4D0022BD
:1010D0000002C01823029B191B0418183B02019C34
:1010E0001B19029C2402039EA4192404E31809C5B9
:1010F0002A606A6008788021814304981346FFF7CC
:0C1100001FFF05B0F0BDC046000000203D
:10110C00F0B585B002AC0DC40C794D792D022C19BB
:10111C008D79CE79360275192D042E198A78CC78F2
:10112C000D7848781A4B00270197DF81000240198F
:10113C002402A218039C1204101841C31C60887965
:10114C00CA79120216180498083B864200D8304619
:10115C009881002E05D0002C0FD100280DD0019CB9
:10116C0012E008788021814300240298224623460D
:10117C00FFF7E0FE002806D106E0029800F00AF81E
:10118C000028019C00D00124204605B0F0BDC046CB
:04119C00000000202F
:1011A00070B504460F48C1898289561AB1B24029E8
:1011B00000D3402600254157002907D5802531045A
:1011C00004D08168B2B2084802F072F8B3B2002BC2
:1011D00001D11A4600E0044A20462946FFF7B0FE36
:0C11E00070BDC046000000208007002009
:1011EC0080B50248142102F065F880BD0000002093
:0C11FC00014908617047C0460000002057
:10120800F0B582B081790191C1790091037944796F
:101218008578C678077841780A4A00200902C919F2
:10122800360275192D0469182402E318009C24025B
:10123800019D64192404E3180AC21060506002B0CA
:08124800F0BDC04600000020CB
:10125000F0B581B01E4604460025294F785741401D
:1012600049B2002918D4002806D4B868002843D011
:101270002549324602F01CF8F8898019F881B968CE
:101280008919B960402E19D3F98880B2814215D0EE
:101290002046FFF785FF23E0002E2DD119480028B6
:1012A00003D01749204600F0EDF83B690125002BDB
:1012B00022D00221124A204698471DE03B69002BAC
:1012C00005D001210E4A2046984700280BD03878D7
:1012D00080218143002520462A462B46FFF730FE19
:1012E000002808D108E00021204600F03FF98021C5
:1012F000204600F03BF90125284601B0F0BDC0466C
:0C13000000000020851400008007002081
:10130C0030B541200006017801220A430270817831
:10131C00C907FCD08178C907FCD116490A68038D2E
:10132C001F24A3435202D20ED21802850A68038DE1
:10133C00114D1D40A301D2091A40521902850968AA
:10134C00028D0E4B134007221203C90A1140C91813
:10135C0001850B49416200210181062101708178D0
:10136C008907FCD4818B828B0A43828308210183F9
:10137C0030BDC046206080003FF80000FF8F0000A9
:04138C004C050020EC
:0C139000014840210160704700E100E0CE
:10139C00034840210160BFF34F8FBFF36F8F70473D
:0413AC0080E100E0FC
:1013B00080B5802100200246034600F007F802486D
:0C13C00001218180018080BD18000041E7
:1013CC00F0B57F270F407801254C2618CD092C014C
:1013DC003251002F244F17D1002A15D1002B13D1D5
:1013EC00224A1778FF09BD421F4F0DD01C4D2A60B1
:1013FC006A681C4D2A4001256D041543184A556036
:10140C00154652683A406A60321949B25468121D46
:10141C0000291749134D0ED42C409B041B09234360
:10142C00136013683B4013600A18137940241C4363
:10143C00147104220DE02C4014600E4C23401468EF
:10144C003C401C4314600A18537980241C4354718B
:10145C0008220818C1791143C1710120F0BDC046A2
:10146C004C050020FF3F00F000C0FFFF04080020E7
:08147C0000010041FF3F0000E8
:101484000878400607D14878052804D18878802157
:101494000143084801700848084901604168084A46
:1014A4000A4001214904511841604168054A0A4033
:1014B400426070470A0000414C05002004080020E7
:0814C400FF3F00F000C0FFFF34
:1014CC0070B588787F2202400B794C792402E3189E
:1014DC001F4D1D40C30940B200240826A640B5424A
:1014EC0006D0641C072CF8D11A4CA5422DD1072428
:1014FC005201194DAD181B01EB185D680726360714
:10150C00B543640764082C195C60144BD218C97875
:10151C0000280AD4032001401078F8230340C8188F
:10152C00401C10700120112109E010788F2303401A
:10153C008807800EC0181030107002202221117103
:10154C00517A01435172012070BD002070BDC0461C
:10155C00FF070000FF0300004C05002000010041C4
:10156C0048B2002801D4102000E020204906090DC3
:0C157C00014A88547047C0460501004138
:1015880048B2002801D4112000E022204906090DA4
:0C159800014A88547047C046040100411D
:1015A400F0B583B01B4C194D28880290E73500270D
:1015B400012001900298F840C0071FD02E78B00790
:1015C4000DD52268019800901148024080203843CC
:1015D400C1B20020034602F001FF02202870F00788
:1015E4000CD0204610380268019E0096084802403C
:1015F400F9B20020034602F0F1FE2E7020352034AB
:101604007F1C082FD6D103B0F0BDC0462000004196
:08161400FF3F0000600500200B
:10161C0070B52B4D2889AE8806400124700706D57D
:10162C000420288100200321224603F0EFF8F00764
:10163C0008D02C8110202881A8800020042122466B
:10164C0003F0E4F8F00607D510202881288000204C
:10165C000521224603F0DAF830071A4E23D508206C
:10166C0028811121298018484268184B1A400325FB
:10167C002D075219426042691A4052194261317069
:10168C0013217172124901604168124A0A406104C7
:10169C00511841604168104A0A40426000200146DE
:1016AC00224603F0C1F8F079C00606D5002008499F
:1016BC00224603F0C9F81120F071FFF76DFF70BDE1
:1016CC0014000041000100414C050020FFFFFF8F7A
:0C16DC0004080020FF3F00F000C0FFFFEA
:1016E80070B504460120C503AA420CD8049D002603
:1016F800E6812572E380A2802160268251004B1E7C
:10170800A3814942618102498A4200D3002070BD09
:04171800018000004C
:10171C00F0B587B005920E460C9FD91B01D24289B9
:10172C00891A82888CB294420BD99D1AACB29C4215
:10173C0002D883899C4201D94389ED1A0582078A14
:10174C0011460B0436D0049002960D980390BC18E9
:10175C007E423D46B618A41ABF1AABB29342F8D2D9
:10176C000F4689B20598814200D30746501B3A1A9E
:10177C000499CD886A4301920597BAB207466F4324
:10178C0000976B430F68F9183B46039F012F13D04A
:10179C00002F52D180B282424BD9009886B2029C63
:1017AC002046324601F07EFDA01904990968019A81
:1017BC0092B240E0002751E080B282423FD90393BD
:1017CC002848009F3A460240029803F06FF8032124
:1017DC00394039D0002006906E43224A1640A2B2FE
:1017EC006A4393190422541A019EB2B2A2423246A1
:1017FC0000D32246039CE318059F1C5C06AD2C54B9
:10180C00401C491E0C06F8D10499096813060BD02C
:10181C000023144606ADED18CE5C2E545B1C641EE2
:10182C002506F7D1C918019EB61A069A02980260CD
:10183C000FE06A43029801F035FD059F0EE0059F0D
:10184C007D43AAB2029807E004980168059F0298AC
:10185C00019E320402D0B2B203F028F8B8B207B03D
:08186C00F0BDC046FCFF0000C6
:10187400F0B58BB0002A09D0C5898788068A047A16
:10188400002C05D097420FD905910BE00026AFE05C
:10189400AE1B01D24489361B0591B91B8CB294420C
:1018A40000D80A46099206E0D21BC4885443091999
:1018B400059135460997791B06952A460E46C9199E
:1018C400ED1B94B2BC42F8D2BA1AC58811466943DA
:1018D40001916C4307900768381904900999881A94
:1018E400029568430390012B89B2089113D0002B11
:1018F400099E76D190B2814231D9019887B2049879
:10190400059C21463A4601F0D1FCE119079800688C
:10191400039A92B227E0009790B2814226D93648C2
:10192400019F3D460540049805992A4602F0E2FFCE
:101934000320384020D005990A682F4604994A5557
:101944000A9204210B1A039DA9B29942294600D395
:1019540019460AAB0128009D13D15A1C2AE02A46D5
:101964004A430498059901F0A1FC3AE0099E2846EF
:10197400704382B2049831E007980068099E039D81
:1019840029E0049BDB19120A5A700AAA921C801ED1
:1019940010D0029B5E43184B1E40A319EB189B1CEE
:1019A400099E079D14781C705B1C521C401E040683
:1019B400F8D101E0099E079D28680B0609D00B4663
:1019C400039D14780470401C521C5B1E1C06F8D145
:1019D40000E0039D6D1A290403D0AAB2059902F010
:1019E40089FF079C20460699089A02F086FDE0814B
:0C19F400B0B20BB0F0BDC046FCFF00001C
:081A000000487047C0450000DA
:081A0800004870475B4D00002F
:081A100000487047834F0000FD
:101A180010B500281AD0052825D8800013490C587D
:101A2800204601F039FC1F2800D31F20002809D0C8
:101A38000F49891C024623780B80891C521E641C9E
:101A4800002AF8D140000B49411809E0074800680E
:101A58000178407800024018054948800548811CF3
:101A68000348018010BD002010BDC0464809002071
:081A7800380800200203000001
:101A8000B0B505460024FEF7CBFD00280BD0FEF7CD
:101A9000CFFD002807D12720C0006843034908185C
:101AA0000079012404402046B0BDC0461404002043
:101AB00080B52721C900414302484018103002F088
:081AC000DBFC80BD14040020D2
:101AC800B0B52723DB0043430648C418204610302E
:101AD80092B202F01BFD0546204602F023FF28467D
:081AE800B0BDC046140400204B
:101AF00070B504462720C0006043094B1E182436E9
:101B000092B2304602F049FD0546304602F0B4FC80
:101B1000402802D3204600F005F8284670BDC04694
:041B20001404002089
:101B2400F0B581B005460024FEF778FD00282CD0DE
:101B3400FEF77CFD002828D12720C0006843144903
:101B44000D182E462436304602F094FC00281CD092
:101B5400A9782046FFF7C2F9002816D0AF1CF83543
:101B640040223046294602F0D3FC3978002809D0B7
:101B7400044600202A462346FFF7E0F9002804D152
:101B8400044602E02046FFF7C1F9204601B0F0BD4B
:041B94001404002015
:101B980080B52721C900414302484018243002F08B
:081BA8007DFE80BD1404002045
:101BB00070B582B02720C100114C204601F080FB97
:101BC0000125258161204002E0800820207300204B
:101BD000E072FF21617100902046103021463831BB
:101BE000402632462B46FFF77FFD009520462430E5
:101BF0007834214632462B46FFF776FD02B070BDA1
:041C000014040020A8
:101C040010B5084C0020207120602046103002F0EE
:101C1400C7FC2434204602F0C3FC0121204602F014
:081C2400CAFC10BD14040020ED
:101C2C00F0B583B0044648790026022842D1887961
:101C3C0002283FD1214B987800283BD18878187026
:101C4C0008780D186878092724280AD1092A08D39E
:101C5C0028783F182D186878242802D1B9B29142FF
:101C6C00F6D905280BD120462946FFF719F900288B
:101C7C0020D0A878114B587028782D183F18687808
:101C8C00042813D168790A2810D12A78981CD91CF9
:101C9C0000910190A918154602222046134602F025
:101CAC00AAFB002806D07E190E3600E03E460348FB
:101CBC0002F036FEB0B203B0F0BDC04614040020F2
:101CCC0070B5137860251D400024202D62D1137946
:101CDC0055792D02ED18304B1E78B5425AD15578F6
:101CEC00203D032D56D8C0467D442D796D00AF4460
:101CFC00010E181E00292ED0012402294AD1294890
:101D0C00002847D0991D002000F04AFD42E0012434
:101D1C0000293FD19D1D072311462A46FFF7F0F9F4
:101D2C0038E0012402291ED0002910D032E0012411
:101D3C0000290CD002292DD1184800282AD09078DF
:101D4C00D17809020918002000F032FD22E011467A
:101D5C00FFF7A8F91EE09C1D072311462246FFF74A
:101D6C00CFF9012416E090781871D17809020E1879
:101D7C0001253540694269412433184602F017FCAD
:101D8C000748002806D00220064072080020294689
:101D9C0000F0FEFC204670BD14040020BD2700009E
:081DAC009D270000AD27000097
:101DB400F0B583B001930F46009042498878C97802
:101DC400002301221E46C41B63426341CD1B6C42A7
:101DD4006C41002E00D01446002C144600D11C4641
:101DE400731C012CEED1002E4DD1B9423ED1354D9C
:101DF400294610312C46B834019882B20291084623
:101E0400214602F0C8FB3049481E814168790246E8
:101E1400FF3A531E9A410A40012A17D10199002919
:101E240014D04D1E2178884209D1029802F032FD67
:101E3400002804D123484179002000F09DFC002DA6
:101E440004D0641C6D1E1F484079EBE71F4800282E
:101E540007D0029802F01EFD002802D1002000F0F5
:101E64005FFC184C204602F05FFDA078B8420AD10E
:101E74001748002802D0002000F086FC0020FFF75D
:101E84004FFE002803D07042704103B0F0BD0D48EE
:101E9400243002F0EFFA01998906F4D1019900295E
:101EA400F1D00028EFD1074881780098FFF716F8A1
:101EB4000028E8D003488178002200981346FFF7F1
:101EC4003DF8E0E7140400207D27000025270000EA
:041ED4008D27000056
:101ED800B0B58C2141430B48401845780024FEF7E3
:101EE8009BFB00280BD0FEF79FFB002807D1002D95
:101EF80005D000202946FFF745F801244440204634
:081F0800B0BDC046F406002044
:101F1000F0B581B01C4600920F468C214143154814
:101F20004518697800263046FEF7DAFF00281ED0F3
:101F300000996E1C002F0AD02F723F2C00D33F2433
:101F400028460930224601F0B3F9641C07E0402C12
:101F500000D3402428460830224601F0A9F908356C
:101F60003178E3B200202A46FEF7EAFF0646304603
:081F700001B0F0BDF4060020F1
:101F780080B502488C2101F09FF980BDF40600204D
:101F880080B502488C2101F097F980BDF406002045
:101F9800F0B585B00F464979002403293BD1134693
:101FA8003A790725554312359D4234D81B4E71782E
:101FB800002930D1049038783818417821292AD15D
:101FC80088210291705001780391731CB11C009113
:101FD8000193039941180323049802F00EFA00288C
:101FE80019D0B879012801D1F879F0700120307141
:101FF800B878307002983058C179007A00024018D9
:10200800F080B178002905D048364023049832463C
:10201800FEF792FF2C46204605B0F0BDF4060020DE
:10202800F0B585B0144613781F221A40012A08D14A
:1020380004902079774A17780025874203D12E46E5
:1020480002E00025D2E0EE43874200D0CEE0F0B2B5
:102058005B069B0F012B1CD0002B00D0C6E000298B
:1020680000D0C2E06378E178062B47D1212945D119
:102078008C214143501888214258002A00D1B5E0EC
:10208800137804982146FFF73DF8002800D0ACE00B
:10209800ACE063785B1E0A2B00D9A7E07B441B7970
:1020A8005B009F4405373EA3A3A3A3A34F5E4A004A
:1020B800002900D099E0A179E3791B025918402939
:1020C80000D340218C234343D3181A460832039285
:1020D800A278E5782D02AF183A0A00253E0600D10D
:1020E80087E0022900D284E00192039A177009332D
:1020F800491E012602961646019A7DE0062B75D1E7
:10210800222973D18C2141435518FFF779FC0246E7
:10211800EB880DE0002968D18C2141435018421DFD
:1021280005E0002961D18C2141435018021D01238B
:1021380004982146FEF7E6FF57E0022924D000293B
:102148001DD052E002292ED000294ED1A179E37981
:102158001B025B18402B49D88C2141435218483246
:10216800E6E7002941D18C2141435218E1785171A9
:102178002A4A002A03D000BF00BF002836D004989E
:102188002146FEF791FF30E08C2141435218A17897
:102198001171214A002A28D0E27812025118C9B2D6
:1021A80000BF00BF21E0A179E3791B02591840293B
:1021B80000D340218C234343D3181D464835A278C9
:1021C800E4782402A418220A260608D0022906D395
:1021D800E6B22F78B74202D14933491E00E02B46B8
:1021E80089B20091E1B200F0F7FA0125284605B05E
:1021F800F0BD039E3346029589B20091F9B200F012
:10220800E1FA029940180104F0D083B204982146FB
:1022180032468FE7F40600200000000000000000AE
:10222800F0B583B0019020484278807800250124D9
:1022380002942F46561A75427541441A6642664101
:10224800002F00D0029E002E029E00D12E467D1C3B
:10225800012EEED1002F01D0002722E08A4209D1B9
:10226800124800281CD010490831DAB2002000F0CA
:10227800BBFA15E0884213D198B200900A4C254663
:1022880048350027384639463A462B4600F0A4FA26
:10229800A178402301982A46FEF74EFE002800D078
:1022A800029F384603B0F0BDF4060020F127000075
:1022B80080B5012807D80A464100034B585C5918D5
:0C22C8004978FDF7E1FF80BDE74F000002
:1022D40080B5012806D84100034A505C511849785A
:0C22E400FDF7E2FF80BDC046E74F0000A0
:1022F00080B5012801D9002080BD4100044A505C0E
:1023000051184978FDF7DAFF411E884180BDC0466B
:04231000EB4F00008F
:10231400F0B589B007AC2046FEF71AF9A3786278C5
:102324002178E078257964790090019502947F48BA
:1023340001F078F8FEF79AF8062801D97C4902E002
:1023440080007C4909587C4801F06CF805AC2046B3
:10235400FEF7B2F80599794801F064F8A188784845
:1023640001F060F8E188774801F05CF8E0880599AD
:102374004143754801F056F8002420462146FEF7F3
:10238400AFF801252846FEF7C1F82846FEF7CEF837
:1023940002212846FEF75AF8284629462A46FEF71F
:1023A4004DF80820049003260096019502902846D3
:1023B40029462A462346FDF7E3FF0095019402943B
:1023C40003942046294622462346FDF77FFF2046F4
:1023D40031462A462346FDF7B3FF092720463946EE
:1023E4002246FDF723FF0A26204631462246FDF702
:1023F4001DFF204639462A46FDF7A8FE20463146F1
:102404002A46FDF7A3FE204639462A46FDF7D2FEAA
:10241400204631462A46FDF7CDFE2046049E31462D
:102424002246FDF703FF0B27204639462246FDF7D7
:10243400FDFE204631462246FDF788FE20463946F9
:102444002246FDF783FE204631462A46FDF78CFEE0
:10245400204639462A46FDF787FE204631462A465D
:10246400FDF7BEFE204639462A46FDF7B9FE204652
:1024740031462A46FDF7CAFE204639462A46FDF76C
:10248400C5FE00F0FBF9FF20000630490A688243CC
:102494000A602F482F49416084600726066028039C
:1024A4002D490A6802430A608868284388602846E0
:1024B400294622462346FDF78FFF69022020FDF7B7
:1024C400A9FF0095019402950394304629463246AB
:1024D4002346FDF7FBFE042031462A46FDF724FF80
:1024E4001727204639462A46FDF7A0FE20463946DE
:1024F4003246FDF7AFFE1826204631462A46FDF740
:1025040095FE1927204639462A46FDF78FFE0625F3
:10251400204631462A46FDF79DFE204639462A4686
:10252400FDF798FE01F055FF09B0F0BDEF4F000034
:102534006750000060250000A64D0000BD43000068
:10254400114C0000B74D0000C44A000020ED00E02B
:0C25540010E000E07F3E0000100400409A
:102560005B500000054C00000B4C00005F50000069
:0C25700063500000A14D0000A5430000D6
:10257C0088B0FFF7C9FE0025012428462146FFF745
:10258C0095FE20462146FFF791FE7D20800000F04D
:10259C0087FA28462946FFF789FE019420462946EA
:1025AC00FFF784FE404800F039FF414F444C474E42
:1025BC0000F06AFA3D490968401AC0087D2806D324
:1025CC0000F062FA394908600020FFF77DFEFEF743
:1025DC008DF8387800280AD1364802F00FF8002818
:1025EC0002D00198387002E03878012811D100F03F
:1025FC0051FA03463048006883420AD02E480360E3
:10260C0002AD142128462D4A02F0B0F8284601F0FC
:10261C00F5FF002007AD294600F078F900281DD001
:10262C00287800281AD12088401C2080012001998C
:10263C00FFF73CFE2188234800F0F0FE3878012893
:10264C0009D1238802AD142128461F4A02F08EF8C6
:10265C00284601F0D3FF002000F0DEF8012007AD82
:10266C00294600F053F90028A2D0287800289FD1E1
:10267C003088401C308001200021FFF717FE318884
:10268C00134800F0CBFE3878012809D1338802AD0D
:10269C00142128460F4A02F069F8284601F0AEFFD3
:1026AC00012000F0B9F883E7D04D0000100800209D
:1026BC0046090020814C00002C080020B34C00007F
:1026CC0080080020264B0000C75000000E08002098
:0826DC00354B0000D75000004F
:1026E40080B5024800F09EFE80BDC046DB4A000073
:1026F40080B5024800F096FE80BDC046E14D000062
:1027040080B5024800F08EFE80BDC046EE4D00004C
:1027140080B5024800F086FE80BDC0466F500000C0
:1027240030B581B0114800F07DFE00242046FFF74B
:10273400BDF9002815D06D46012220462946FFF731
:10274400C1F9002801D02D7800E0E5430848294666
:1027540000F068FE782D02D10120FFF7B9FD0020BA
:10276400E5E7044800F05EFE01B030BDE64A000033
:08277400FB4D0000F54A0000D6
:10277C0080B5024800F052FE80BDC046274C0000D8
:10278C0080B5024800F04AFE80BDC0467B50000078
:10279C0080B5024800F042FE80BDC046F84A0000F9
:1027AC0080B5024800F03AFE80BDC0469350000050
:1027BC0080B5024800F032FE80BDC0460F4B0000D1
:1027CC0080B50348029A00F029FE002080BDC04667
:0427DC003D4C000070
:1027E00080B50248029A00F01FFE80BD5F4C0000D9
:1027F00080B5094800F018FE08490878002809D07B
:102800000020087001460246034601F0E2FE04483B
:1028100000F00AFE80BDC046AB500000F307002068
:04282000004E000066
:1028240030B583B0044600252846FFF753FB002843
:102834001ED01048017800291AD101AB5D712D21F9
:10284400D97011219970172159700521197001212E
:102854000170002C01D01F2000E01E2018712846B2
:1028640029462A4601F0B3FE611C034800F0DAFD54
:0C28740003B030BDF3070020BD4C000095
:10288000F0B581B000200125094C8700E619C0B2DF
:10289000FFF72EFDB070B078002800D01920E0536B
:1028A0000021F1700120EA070D46EED101B0F0BD24
:0428B0007808002084
:1028B400F0B581B000200121154C0D468700E619C2
:1028C400C0B2FFF713FDE15B00280BD0192918D023
:1028D4003188491C31803188192912D1B1780129F4
:1028E4000BD10EE000290CD03188491E318031888B
:1028F400002906D1B178002903D0B11C0870012049
:10290400F07001200021EA07D7D101B0F0BDC04624
:04291400780800201F
:10291800012801D9002070478000064A121872B6B3
:10292800D0780023D37092780A70411E884162B62D
:082938007047C046780800203A
:0C294000014800F071FDFEE7E7500000C8
:0C294C00014800F06BFDFEE7194E000092
:0C295800014800F065FDFEE7264E00007F
:0C296400014800F05FFDFEE7334E00006C
:0C297000014800F059FDFEE7D74C0000C4
:0C297C00014800F053FDFEE7444B000052
:0C298800014800F04DFDFEE7404E00004D
:0C299400014800F047FDFEE7514E000036
:0C29A000014800F041FDFEE7624E00001F
:0C29AC00014800F03BFDFEE7734E000008
:0C29B800014800F035FDFEE7844E0000F1
:0C29C400014800F02FFDFEE7954E0000DA
:0C29D000014800F029FDFEE7E54C000086
:0C29DC00014800F023FDFEE7F34C000072
:0C29E800014800F01DFDFEE7014D00005D
:0C29F400014800F017FDFEE7A64E0000B1
:0C2A0000014800F011FDFEE7B34E00009D
:0C2A0C00014800F00BFDFEE7C04E00008A
:0C2A1800014800F005FDFEE7CD4E000077
:0C2A2400014800F0FFFCFEE7F750000046
:0C2A3000014800F0F9FCFEE7DA4E00005F
:0C2A3C00014800F0F3FCFEE7E74E00004C
:0C2A4800014800F0EDFCFEE7F44E000039
:0C2A5400014800F0E7FCFEE70F4D000019
:102A600009480188491C01807D22D20089B2914227
:102A700005D10021018005480168491C0160044816
:102A80000168491C0160704782080020300800205E
:042A900034080020E6
:0C2A9400014800687047C046340800206C
:0C2AA000014800687047C0463008002064
:102AAC0003490A680B689B1A8342FBD37047C046E4
:042ABC0034080020BA
:102AC0000122D20703004B403DD430B4431A01D257
:102AD000C01AC9184B004400240EFF2C29D0002C2A
:102AE00024D01B0E20D0E31A182B1DDC0902114341
:102AF000C40D000210435D4219350A00AA40D209F4
:102B0000D940451801D36D080234013CE405280A78
:102B10000121C9072D062A438A4160414100090E5F
:102B2000FF2901D3C00DC00530BC7047C00FC007DE
:102B3000FAE742001823DA41FF2AF5D07F2000018E
:102B40000C300005F0E7A4465140431A02D253402E
:102B5000C01AC9184B00090211431B0E4400240E71
:102B6000FF2C41D0002B10D05B421B19012B10D33E
:102B700022D1C30D4002401A10D3DB050100400AE8
:102B8000C90591415841644670472442FBD1002059
:102B9000F9E7C30D40024900401AF4D00021013189
:102BA0004000FCD38C4204D95B1ADB05400AC018F4
:102BB000E9E7180AC007E6E7192BE4D801330C004F
:102BC000D940DC414C40012C4941C30D0002104367
:102BD000441A01D4A4006408013BDB05200A240642
:102BE0009441584164467047FF2B01D04102CAD03E
:0C2BF0007F2000010C300005C5E7C04646
:102BFC000122D2075140014B18470000C52A0000A2
:102C0C0030B405004D400124E407254042004B0040
:102C1C00120E32D01B0E3CD0FF2A33D0FF2B3FD0EC
:102C2C00D21800022043000A09022143090AC4B247
:102C3C004C43000AC3B24B43000A4843210A5B18B9
:102C4C00190A091801D44900013A080A7F3A2ADB0B
:102C5C00FE2A0FD2D2051C43240601D001242143A5
:102C6C00C9B280295041802901D140084000284335
:102C7C0030BC7047FF20C005F9E71B0EFF2B0AD0B4
:102C8C002800F5E7400206D1FF2BF3D1490202D10F
:102C9C00F0E7FF2AF4D17F2000010C300005E7E7B4
:102CAC004902F8D1E6E743020132E9D15B12023363
:082CBC00E6D9D805E4E7C046A3
:102CC40030B405004D400124E407254042004B0088
:102CD400120E26D01B0E34D0FF2A2DD0FF2B35D058
:102CE400D21A000220430902214343084908A00DD7
:102CF4005B1A02D2013A5B005B185B008B4200D383
:102D04005B1A4041F9D37F3222DDFF2A06D2D20575
:102D1400C91A8B425041284330BC7047FF20C0057C
:102D2400F9E71B0E03D0FF2B12D1490210D07F20EC
:102D340000010C300005EFE74002F8D1FF2BEDD184
:102D4400F5E7FF2AEAD14002F1D1E7E74902EED1E3
:042D54002800E1E78B
:102D580002000A43520008D0884204D140000121F1
:102D68000906C84201D90020704701207047C046B3
:102D7800012212064300DA4211D84B00DA420ED87B
:102D880002000A43520008D003D288428041013031
:102D98007047814280410130704701207047002010
:042DA8007047C0466A
:102DAC00012212064300DA420FD84B00DA420CD84B
:102DBC0002000A43520008D003D2814280414042B3
:102DCC007047884280414042704700207047C0469F
:102DDC00012212064300DA420FD84B00DA420CD81B
:102DEC0002000A43520008D003D28842804140427C
:102DFC007047814280414042704700207047C04676
:102E0C00420017D2120E7F3A14D480231B06202ABC
:102E1C0006DA52421F3200021843D040002170479C
:102E2C0052423F3209DB010219430800D041D14024
:102E3C0048407047002001007047D01701007047D0
:102E4C009D2201000AD002D4013A4900FCD5D205DA
:102E5C00080A0906494100D3012950417047C04670
:102E6C00BD22094210D003D4013A00184941FBD5C8
:102E7C00D2050128804101300143080A0906494165
:102E8C0000D3012950417047004908474D2E0000DE
:102E9C004B1801225205DA4217D25B0D0722D201E0
:102EAC009B1A0FD9FF2B13D2DB05CA0FD207134382
:102EBC000903020D1143490AC200524100D90131E4
:102ECC00C8187047C80FC007704706D1002804D136
:102EDC00C80F0002FF30C00570470123DB070A0052
:102EEC00C900400F084398431A4010435B0A18432B
:042EFC007047C04615
:102F0000F0B583B00C460191394AC10D4B1EFD2B23
:102F100048D8FD23DB43E50DFF3D9D4242D30346E8
:102F200013402646541C04400293B3424ED9CDB2FE
:102F3000324F002D04D03840791C0143029104E047
:102F400002A8002101F094FB0546F00DC0B2002854
:102F500003D03E40791C314304E001A8002101F078
:102F600087FB0199029A854208DD531A01D41A465B
:102F700015D06D1E52008542F7DC05460292501AAC
:102F800001D40CD0029002A8294601F071FB01285F
:102F90001FDBC0051A494118029800194418204641
:102FA00003B0F0BD4500134B9D4210D26500AB420B
:102FB000F5D903461340FF25EE050F4DB34214D05B
:102FC000002B0CD114420446E9D10EE0E7D00446B0
:102FD000E5E70121091A0298C8400021DDE7144005
:102FE00003D0B442F3D001949BE72C46D7E7C04608
:102FF000FFFFFF7F010000FF0000C07FFFFF7F0099
:04300000000080FF4D
:10300400C10DC9B24A1EFE2A19D27E2903D800284E
:1030140013DA1048704795290ED87F390C4A0A41B3
:103024000240134603D5094B5B1CCB40D3188840A0
:10303400400200D01A46104670470020704700290D
:10304400FAD10121C90708407047C046FFFF7F003D
:08305400000080FF000080BFB6
:10305C0030B5514343435C18010C130C0D005D4318
:10306C00641992B2514380B242430D0C09045218B8
:10307C0065415843010C00048018694130BDC046BD
:10308C00CA1751408B1A17D0C1174A409446484072
:10309C00411A48081A0000E052008242FCD9002074
:1030AC0000E05208914200D3891A40419A42F8D16B
:1030BC0062465040801A704710B500F07DF810BD84
:1030CC0007B5FFF7DDFF0EBC4243891A00BDC046B1
:1030DC000A0015D00300400800E052008242FCD9DF
:1030EC00002000E052089B1A06D340418A42F9D1D5
:1030FC00704752089B18F8D200188A42F9D17047D1
:08310C0010B500F059F810BDE8
:1031140038B504004D42FFF7DFFF4543611938BD60
:10312400002B09D1002907D110B51100FFF7F0FFDA
:103134000A000021002310BD70B400240125ED070E
:10314400002B07D1002905D0834203D213000022AB
:103154002C0000250026A419994200D1904212D9CE
:1031640092185B4103D2EE076D086408F3E7DE07AB
:103174005B08520892190126F6079B1903E0DE0743
:103184005B0852089219801A994103D364416D4136
:10319400F5D30FE024196D410AD2DE075B0852080B
:1031A400921980185941F5D364416D41E7D301E088
:1031B4008018594102000B002000290070BC7047A0
:0831C400002000217047C04605
:1031CC0003490868002800D070470248086070471F
:0831DC0014080020780900200E
:1031E4007F2805D8034A125C0348405C10407047AE
:0C31F4000020704703510000624F0000F3
:103200007F2805D8034A125C0348405C1040704791
:0C3210000020704703510000624F0000D6
:0C321C001D4D0000483200002832000068
:10322800E5310000514A00005D4A0000013200000B
:10323800694A0000754A0000414A0000154A00002A
:103248001F4D00004F4F00004F4F00004F4F000030
:103258004F4F00004F4F00004F4F00004F4F0000EE
:103268004F4F00004F4F0000FFFFFFFFFFFFFFFF22
:10327800FFFFFFFFFFFF0000214D0000014F00008E
:10328800534B00001E4F0000AA4B0000504F000097
:08329800594F0000B14B00008A
:1032A000411C02780130002AFBD1401A7047C04609
:1032B000002A03D0013A8B5C8354FBD17047C0468F
:1032C00000220B0011001A00002A02D0013A81549A
:0432D000FCD1704776
:1032D400F0B581B00022002933D00378002B30D020
:1032E400032302469A4316680024E5438707FF0E2A
:1032F400BD40ED43354306461E4071180429009332
:103304000AD3124EAF19104BAB433B4204D1091FF1
:103314005568121D0329F5D82B060DD02B041B0E5E
:1033240007D02B021B0E06D02B0E009C04D00424C5
:1033340002E0012400E002248C4200D82146101A45
:103344004218104601B0F0BD80808080FFFEFEFE72
:10335400F0B581B00446C017271847407F20C50543
:10336400002F00950BD0C505094EF80704D031682D
:103374002846FFF749FC0546361D7F08F5D100981D
:103384002946FFF79DFC002C00D4284601B0F0BD6F
:04339400983300006A
:10339800000020410000C84200401C4620BCBE4C32
:0833A800CA1B0E5AAEC59D744C
:1033B000F0B503AF93B06E46F51D2135F41D3934D9
:1033C00074613362F261F160306100F0FDFEB06063
:1033D000C21D07218A436946B1616946881A706037
:1033E0008546F41D1D34002124222046FFF76CFF82
:1033F0000B487169F2680A6048600A4828603069C1
:103400002862B06868617068E8602046F169326AD5
:1034100000F01EF8B1698D46FC1F053CA546F0BDC5
:08342000B54A0000FFFFFF7F29
:1034280083B010B581B0044603A80EC005480068F3
:1034380003AA0092214601F0B4F901B010BC02BC05
:0834480003B008478C090020C5
:10345000F0B59FB014460F46002115900160012081
:1034600002020C92460282020392C20202920322DC
:103470000A92920205920203179242030792820374
:1034800004920090C00316900891C84301901096D2
:103490003978252908D0002901D100F063FE7F1C6E
:1034A000159801F00AF9F3E7FF1C089BB81E057890
:1034B0002A46203A102A2BD880219200184602A3CF
:1034C0009A5803469746C0460D3500002D3500003A
:1034D0002D350000273500002D3500002D3500006A
:1034E0002D350000193500002D3500002D35000068
:1034F000553500001D3500002D3500002135000038
:103500002D3500002D3500002535000040210AE052
:103510005E2D179907D009E0169904E0202102E0FA
:10352000102100E031460B437F1CBFE77F1E294678
:103530003039C9B20020092919D80A214143681835
:103540003038791C3D782A46303AD2B20A2A0F46E2
:10355000F3D30AE001CC002801D510210B43C11799
:1035600042184A40781E05781046C11788432E2D10
:1035700008D13D782A2D08D17D78BF1C214610C97D
:103580000F9116E000210E911EE07F1C2946303974
:10359000C9B2092912D80F9400240A2161436C187A
:1035A000303C791C3D782A46303AD2B20A2A0F467E
:1035B000F3D30E94002C0F9C02D505E000210E9150
:1035C00001460C980343084629466839CA01C9B226
:1035D00049085118C9B2092926D8C0467944097941
:1035E00049008F44040A112121210E21210E3D782A
:1035F000682D13D1014608200BE001460220034349
:1036000008463D787F1C0FE03D786C2D09D10146BE
:103610000220034308467D78BF1C05E07F1C04217F
:1036200001E07F1C01210B43462D0B9025DD29462F
:103630006339152934D849007944898849008F4471
:103640004F0016004B002600BD01150016001500A6
:1036500015001500150061006C00790015001500BB
:1036600087001500890015001500370010E7049841
:10367000034300210991194675E0442D159808DD92
:10368000452D27D0462D00D002E707980343029826
:1036900023E0252D00D06BE2252101F00EF8F7E69E
:1036A000472D00D188E1582D00D0F1E6079803435B
:1036B000614A782D00D120321906C81709900C985C
:1036C000034201D05D48034019460498099B13400A
:1036D000099348E00798034303980343059A6FE171
:1036E000264624780B98421E159D284619461392AB
:1036F000149301F036F82846214600F0DEFF1498B6
:10370000341DD4E1180700D536E2980700D58FE2C2
:10371000159800682168086090E20C9803421946E9
:1037200001D0464801401A06D217302010400990B7
:10373000049818E0069718060C990B43C01723212C
:103740000140099104CC0F94002708200E90D0E08E
:1037500001CC82E10C98034201D03848034019465D
:1037600004980022099202220A400142069706D1DB
:10377000002A09D1231D002722461C460AE0002A00
:1037800012D104CCD01715E0E21D07239A435768E5
:103790001446083413684A0718D408220A4000D097
:1037A000DBB2002A13D128E0E41D072294432268EB
:1037B000606808344B070CD408230B4000D0D2B209
:1037C000002B00D000200746134605E09BB20027DF
:1037D00013E013B21204D717002F05D48A060AD4B7
:1037E0004A060AD5202007E000225B42BA412D207C
:1037F0000990174601E02B2009900C981A460142C7
:1038000001D00E4801400B460C9801420F9401D1A3
:1038100001200E9000246E2D2ADD6F3D092D00D968
:1038200088E0C0467D442D796D00AF4409628383F2
:10383000838327838362C04658300000FFFDFFFF6B
:103840001046384376D0D008790740180024014646
:1038500007201040303018AA1055C808FF087A0712
:1038600080180A463A43641C002A0A46EFD161E0F8
:10387000582D3ED0642D01D0692D5BD110463843C0
:1038800058D01946169801400D9100211493144602
:103890003B460D9800280AD00F4608460A99084072
:1038A000032805D118A82C21C1557F1C00E00F4624
:1038B0000A26002520461946324613932B46FFF769
:1038C00031FC11940446129132462B46FFF7C6FB99
:1038D000119A101A3021014318A8C155791C0920EA
:1038E000801A13988541129F109E149BD0D30C46CA
:1038F00020E0104638431CD007981D460342E84894
:1039000000D0E848134611093A07891800240A46EE
:103910000F211940415C18AB195511093F093B07AC
:10392000C91813463B43641C002B1346EFD12B46AA
:1039300000E00024099A511E104688410B99091B8A
:10394000FF2A00D9491E069F081A0E990D1BE91778
:103950008D43421B3342149304D11598194600F04D
:1039600000FF0022099E310A139203D0159800F03F
:10397000A4FE139A002E3146159E03D0304600F067
:103980009CFE139A3046149900F0EBFE302130462D
:103990002A4601F075F8012C0ADB641C18A80019EE
:1039A000801E0178304600F088FE641E012CF5D898
:1039B0001498C0060F9C7BE007980343059A1343B5
:1039C0000C98034201D00E9800E006201493134097
:1039D000991A4A424A41002800D002460E92E41D3C
:1039E0000720844303CC083CFFF758FA25460446D9
:1039F00000F037FE08350F9500280FD00021204633
:103A0000FFF7ECF9149B1A4607990A40002814D0D6
:103A1000002AE6482C461ED0E5481CE0204600F06F
:103A200017FE00284DD00798149B0342E14800D0B0
:103A3000E148E2490B400F9C0FE0002AE0492C4688
:103A400000D0E049002A01D0DE4800E0DC48401CFC
:103A50009A0600D50846D9490B400028DA4E00D016
:103A600006461946D948014014910C9803420F9418
:103A7000304602D1FFF714FC02E00E99FFF72AFC52
:103A800005460B98421B1598149C2146139200F092
:103A900068FE002D09D0159C3178204600F00DFEFF
:103AA000761C6D1EF8D1149800E020460F9CC006CD
:103AB000109E00D4ECE420211598139A00F0E0FF4A
:103AC000E6E40126204600F071FF0546002801D0FB
:103AD000F007444013961EA9204600F085FF1E986B
:103AE0000A9948430A21FFF7D1FA06461E90602141
:103AF000002D0D9102D01498084314900025204603
:103B00002946FFF729F900281AD1701CFFF722FC7B
:103B100001462046FFF74AF9002804D01E98411CB0
:103B20001E91801CF2E71E98FFF714FC0146204608
:103B3000FFF754F9002803D01E98401E1E90F3E7AB
:103B40001295149A16460598064013998D02AE42B6
:103B500017D086420E9B06D11E98834212DD0421A7
:103B6000C94388420EDD0398024213D112933CE10F
:103B7000002D00D08CE405E32068159909680170D8
:103B80005CE01E98262811962ED120469049FFF71A
:103B900099F82FE01E98C1435E18102E00DB102606
:103BA0000E2800DD21E11498000600D51CE1002E4E
:103BB000129600D119E13046FFF7CCFB2146FFF702
:103BC00025F83F210906FEF77BFFFFF71BFA814925
:103BD000FFF796F900211291FFF7BEF8002800D1F7
:103BE00002E1761EE7D100E14042FFF7B3FB214638
:103BF000FFF70CF80446774D00211291FFF7ACF85F
:103C0000002845D1204600F02CFD002819D00021C5
:103C10002046FFF7E3F8149B1A4607990A4000284C
:103C200000D18DE0002A61480F9C00D0F4E612E735
:103C3000206800214160159909680160241DFFF783
:103C400027FC20462946FFF797F81E9E00280BD038
:103C500020462946FFF736F804462946FFF78CF838
:103C6000761C0028F4D11E967F20C50520462946E3
:103C7000FFF7B4F800280BD020465649FEF7C6FFE0
:103C800004462946FFF7AAF8761E0028F4D11E96AE
:103C900005981199814207D00E98064606E0C04665
:103CA00093510000835100000E98461E019D00288C
:103CB00000D106467042FFF74DFB294600F078FE22
:103CC0002146FEF7FDFE0546424C2146FFF754F81B
:103CD000002807D01E98401C1E9028462146FEF75B
:103CE000F1FF0546149A002E0D9530D00299084632
:103CF00080301040884229D1102E00DB1026344637
:103D00003046FFF727FB2946FEF780FFFFF77EF8D6
:103D10000E46014631431AD0314605462E4A2F4BF6
:103D2000FFF79CF94A08C3079A184008C907081802
:103D30002B49081A2B48904100D3FBE1129406E06E
:103D4000002A1F490F9C00D07BE67BE61296129B4F
:103D5000002B0098149A01D1D0B2C0090B99C91A4E
:103D6000081A451F1E9C17980242139E02D11196F5
:103D70001299B6E0032120461191FFF7A7F9881C9C
:103D8000042800D9A5E0C046784400794000874463
:103D90000297A2029700641E1E940D98FB49FEF73D
:103DA00035FF0D906D1E022096E0C046744F000056
:103DB0006F4F0000A7510000A3510000FFFEFFFF5E
:103DC0007E4F0000794F0000C04B0000FFFDFFFF59
:103DD0009976967E00002041CDCCCCCCCCCCCCCCFE
:103DE00099999999999999191296129840421E9900
:103DF0001039814200DB0846FFF7ACFA019900F068
:103E0000D7FD2146FEF75CFE04461E98401CFFF7D6
:103E1000A1FA01462046FEF7C9FF1E99002800D0EE
:103E2000491C0029149811D4112914D308461038BC
:103E30001E901020401AFFF78DFA2146FEF7E6FE8D
:103E4000FEF7E4FF06460C46002012E0139400261D
:103E50001E9634460FE000201E902046FEF7D6FF47
:103E6000139406460C46FFF701F801461398FEF737
:103E7000C5FE13901498A843C649083100250A4688
:103E800008326D1C0B684968F31A23468B411146B2
:103E9000F6D21195129B002B0099149A01D1D1B240
:103EA000C9090D9D2A4001D00022D243511A1E9A01
:103EB000891A0B9AD21A5118119A891A024632E0BD
:103EC000A41E1E940D98B249FEF7A0FE0D90AD1EE3
:103ED00003E0002000E001201190149A1299C81705
:103EE00081435006800F129100D06D1E0E95F50291
:103EF000204600F08BFD632802DD0E98401E0E90D8
:103F000014980D9CA84314902046FEF77FFF254689
:103F100006460C46FEF7AAFF01462846FEF76EFE4F
:103F2000149A13900E99C8170D46854310981030B7
:103F30000242149209D1012907DB2021159800F0D3
:103F4000BCFB6D1EF9D10025149A4020104091064B
:103F500003D400280AD0202104E0002801D02D211C
:103F600000E02B21159800F0A8FB149AD0060AD483
:103F7000002D08D03021159800F09FFB6D1EF9D15F
:103F800000200E9000E00E951199491E0D46C800C4
:103F9000804A111849681258B01A2046884101D247
:103FA000302007E03020B61A8C41401CB31A23465B
:103FB0008B41F8D2C1B2159800F07FFB2946002D45
:103FC0001498E2D10146029801401191159E0BD040
:103FD0001E98012808DB401E1E903021304600F05C
:103FE0006CFB1E980028F6DC802014990840129C77
:103FF00020430E9D4BD02E21304600F05EFB102C4E
:10400000264600DB1026F01734468443119800281A
:1040100001D1204601E01E98201AFFF79BF90146C6
:1040200012981194001B0D90012E23DB1398FEF7BC
:10403000EDFDFEF7EBFE04460E46119B5B1ED8001D
:10404000544A111849681258A01A304688411393EF
:1040500001D2302007E03020A41A8E41401CA31A60
:1040600033468B41F8D2C1B2159800F026FB139B62
:10407000002BE3D10D980028159E129807D01199B6
:104080000C1A3021304600F018FB641CF9D3039859
:10409000149901423ED00798014201D0452100E029
:1040A0006521159C204600F008FB1E98002805D4C9
:1040B0002B21204600F001FB1E9806E02D21204612
:1040C00000F0FBFA1E9840421E90642810DB642426
:1040D0002146FFF703F801463031159E304600F0C7
:1040E000ECFA1E982146FEF7F1FF08461E9100E00B
:1040F000159E0A242146FEF7C9FF0146303130469D
:1041000000F0DBFA1E982146FEF7E0FF3031304622
:1041100000F0D3FA002D0F9C109E01D1FFF7B8F9E3
:10412000159C2021204600F0C8FA6D1EF9D10F9C85
:10413000FFF7AEF9129428460A2500231193314661
:104140002A46FEF7EFFF04460E462A46119BFEF76D
:10415000E9FF1298401E129000D1F8E51A4320465C
:10416000EAD0F4E5159CE068002805D006CC083CB0
:10417000914201D2089A4254204600F0E5FA2068A4
:104180001FB0F0BD00F0E0FA0198F9E7000020410F
:084190000000C842B00000006D
:10419800084B1B6883420AD0074B1B68834206D032
:1041A800064B1B68181A431E98414042704700206E
:1041B800FCE7C046900900208C09002094090020E3
:0441C80040207047DC
:0C41CC0010B5006800F0CAF810BDC04635
:1041D80003231048104A03614361104B8261C36195
:1041E8008023DB000362002383624362C3620266AA
:1041F8000B4A53214266102282660367094AC36646
:10420800436700E0D17BC1540133013A102BF9D147
:104218007047C0464C0600209C4300001400002054
:08422800F4070020AC43000084
:10423000F8B54746CE46C56883680400406899468D
:104240005B1B80B50E00170098464019934207D9B2
:10425000FFF72EF8ED19E560C0BCB946B046F8BDD1
:104260001A00FFF725F84B463100ED19ED1A2A0028
:0C42700060684144FFF71CF8EDE7C04611
:10427C00F8B54746CE46002380B5884607001600A1
:10428C009946C56884681BE0013B5B1B641BB44208
:10429C0000D934009C4200D91C00786822004146A9
:1042AC004019FEF7FFFF2D19A144A044361BBC6832
:1042BC00631B5A1E93415B421D40FD60002E06D0CD
:1042CC003B699D42E0D3013B1B195B1BDEE7484673
:0842DC00C0BCB946B046F8BDB4
:1042E40070B50600431C5C00E418E00074001C4B2D
:1042F400A419E400C0181B19DC6A1500012C06D0AF
:10430400022C1FD0002C10D00024200070BD9A6A0B
:104314005C6AA2421FD9013A121B2C00954200D9B3
:1043240014002200FFF782FFEFE79A6A5E6AB24246
:104334000CD9013A961BB542E7D82A00FFF776FF5D
:104344002C00E2E7FFF798FF0400DEE71B6AD218AF
:10435400013A961BEFE71B6AD218013A121BDCE7FD
:044364004C060020E3
:10436800F8B50B4B04001B780D001600002B0CD081
:10437800EFF31087012181F3108832002900200013
:10438800FFF7ACFF87F31088F8BDFFF721FFEFE7D1
:044398004C060020AF
:09439C005465726D696E616C00DC
:0743A5004241434B5550005B
:1043AC00000000000000545452205245474745532A
:0143BC000000
:0F43BD004E564D2070616765733A2025750A00D2
:0243CC00FEE70A
:0243CE00FEE708
:0243D000FEE706
:0243D200FEE704
:0243D400FEE702
:0A43D60080B50020FCF737F980BD28
:1043E00030B583B06C4607256570207000200190C1
:1043F00021716371029206992046FCF7E1FC03B03B
:0244000030BDCD
:10440200F0B585B004930124002A23D015460E4648
:10441200074601940B9803900A9802907078002442
:10442200052817D1F078032101400498814211D167
:1044320038463146FCF739FD00280BD002203056B1
:104442000028039900D402990870307836186D1E3E
:0A445200E4D1019C204605B0F0BD46
:10445C0070B514460D460646C868FCF7C9FEEB68F5
:0A446C00002130462246984770BD3B
:0244760070478D
:10447800C189028A891A01D24289891A8AB2808836
:0A448800824200D3014688B270475B
:10449200B0B50446C289038A00F009F80546218AAC
:0E44A20020462A4600F02AF820822846B0BDA7
:1044B00070B5D41A01D24589641B8588A6B2AE4274
:1044C0000AD9541BA6B2964202D88289964201D9D3
:1044D0004289A41A04822C4622040CD05A1B9EB294
:1044E000AE421346FAD2C288564300688319084682
:0E44F0001946FEF7DDFEA0B2411E884170BDE8
:1044FE00521893B28B4202D381898B4201D94089E3
:06450E00121890B2704784
:0A45140080B5002300F001F880BD1F
:10451E00B0B582B00446C589008A0090019320464A
:10452E002B46FDF7F4F80546218A20462A46FFF76A
:0A453E00DFFF2082284602B0B0BD66
:1045480070B50446C589008A2A1A01D26089121AF0
:10455800A08892B2824202D1227A002A17D02A4633
:10456800161A93B283423246FAD2E288534320683D
:10457800C018FEF799FE681C81B2A94202D3A2892D
:10458800914201D961894018E081012070BD002065
:0245980070BDF4
:0A459A0080B50023FDF769F980BD2C
:1045A4000021C1810182818849004A1E82814942D9
:0645B40041810120704767
:0645BA00017201207047B0
:1045C00012010002EF020140FECA010000010102D7
:0245D0000301E5
:1045D20030B583B00C46054601A800214170027037
:1045E200801C002B04D006221946FEF760FE02E072
:1045F2000621FEF764FE01AA082328462146FDF79C
:0646020086FC03B030BD90
:1046080070B5044600252846FDF736FA002814D070
:104618002846FDF7BDFA06462046FEF73DFE8642CF
:104628000BD32046FEF738FE024628462146FDF702
:0E4638005BFA2846FDF772FA0125284670BD90
:0A46460080B50020FCF7E7FF80BDFF
:10465000FF2109064000884201D800207047012050
:024660007047A1
:0E4662000121090640004118484248417047B6
:10467000F0B50268140C01D0134600E013041E0EBE
:1046800000D11B021D0F00D11B01674267413C0195
:10469000002E00D108349E0F002D00D1241D002EC5
:1046A00000D1A41C002E00D19B00DB43DB0FE318DC
:0A46B000083B9A400260C81AF0BDF2
:1046BA0030B581B0044668460170206900280FD0E1
:1046CA000CCC083C9A4235D26269531C636181540E
:1046DA00A069616981422DD1204600F030F829E0B5
:1046EA00E06800280BD00CCC551C083C9D4202D136
:1046FA006D46002129709A421CD281541AE0A068A2
:10470A00002808D00CCC083C9A4213D2551C9D4272
:10471A000DD0C9B20CE0236A002B0BD003CC083CA5
:10472A00884207D2694601222046984702E00021C2
:0E473A00920081502068401C206001B030BD0C
:1047480010B54269002A07D00446036A002B01D03D
:0A475800216998470020606110BD40
:1047620080B5CB0606D4890501D5302100E0202191
:0647720000F085F980BD96
:1047780081B0F0B58AB014460D4606460F930FA8CF
:10478800009001AF384600F085F902950496009A2A
:1047980038462146FEF758FE0AB0F0BC02BC01B00C
:0247A8000847C0
:1047AA0070B514460D460646FEF70BFD0146304627
:0A47BA002A462346FEF7F7FD70BD06
:1047C40008001000200040008000000100020004E6
:0C47D4000820006800BF00BFFBF7EAFEF1
:0847E00080B5FBF72DFF80BD41
:1047E80030B5002A0DD08A184C78052C05D18C7864
:1047F80065062D0E4519E4092B550C7809199142C7
:04480800F2D330BDFA
:0C480C0080B5FCF7FFFBFCF7EBFC80BD67
:1048180000B583B06B465970187000200290019063
:0C48280018461146FCF7C8FA03B000BDAA
:1048340010B584B001AB01245C70187000200290A4
:104844001971039018461146FCF7B8FA04B010BD6C
:1048540030B583B0034668460624447003700B7970
:104864004C792402E3188C79CD792D022C19240477
:10487400E31802930B784C782402E3188C78C978F7
:10488400090209190904C91801911146FCF796FA9D
:0448940003B030BD80
:0C489800C189008A091A48424841704753
:1048A400C189028A891A828801D24089091A501A58
:0448B40080B2704717
:1048B80070B582B0044690080ED00B784D782D0262
:1048C800EB188D78CE78360275192D04EB18236015
:1048D800091D401E0304F0D10320024006D0002029
:1048E800019001A8FEF7E0FC0198206002B070BDBD
:1048F80030B581B093080BD00C680470250EC570D4
:10490800250C8570240A4470001D5B1E1C04F3D11D
:1049180003231A4004D0096800916946FEF7C4FCD5
:0449280001B030BDED
:10492C00B0B50446054610352846FFF7B5FF4028BC
:10493C0015D3E1780020FCF7CDFA00280FD02846DB
:10494C00FFF7AAFFE178402806D3B83400204023B3
:10495C002246FCF7EFFAB0BD0020FCF7D3FAB0BD4D
:0C496C0080B5FEF777F8FDF79FFF80BDD7
:10497800F0B581B01E4615460C4607461846FFF7A7
:1049880007FC0146002000290AD46543A54207D345
:10499800304639462A46FFF715FC2146FEF79AFBB2
:0449A80001B0F0BDAD
:0449AC00C00F704781
:1049B00010B5FD22D343C20DD2B21446FF3C9C4237
:1049C00011D351184A1EFD2A05D8FF22D205904363
:1049D000C905084310BD0122D2071040012902DB9E
:0849E000FF21C905401810BDBC
:1049E800C20DD2B2FF2A01D0002A02D100220A60E9
:1049F80070477E3A0A60FF21C90588433F210906AE
:044A0800401870479B
:084A0C00C11740184840704733
:104A140010B5002A0DD00446097848B200280AD4FB
:104A2400002C00D02160002119605960411E88418A
:0C4A340010BD002010BD0120C04310BDCB
:104A4000024601207F2901D9C04370471170704789
:0C4A5000014661391A2900D22038704755
:0C4A5C00014641391A2900D22030704771
:0C4A6800014661391A2900D2203870473D
:0C4A7400014641391A2900D22030704759
:104A800070B5012A09DB0C460546561C284621460E
:0C4A9000FFF713FE761E012EF8D870BD53
:104A9C00B0B50446FEF794FB0546002124222046BF
:084AAC00FEF70CFCE561B0BD52
:104AB40010B50C46436A01212046FFF75BFF10BD89
:104AC400466C6173682073697A653A2025752062A3
:074AD400797465730A0A0002
:0B4ADB00555342206D6F756E740A0089
:0F4AE6007475645F6364635F72785F63620A0074
:034AF5000D0A00A7
:104AF8007475645F6364635F6C696E655F7374612A
:074B080074655F63620A009F
:104B0F007475645F6364635F73656E645F6272651F
:074B1F00616B5F63620A0095
:0F4B2600427574746F6E2031205B25755D0A0037
:0F4B3500427574746F6E2032205B25755D0A0027
:0F4B44002A20495251204556535953202A0A001E
:104B53004A616E7561727900466562727561727938
:104B6300004D6172636800417072696C004D617938
:104B7300004A756E65004A756C79004175677573F7
:104B8300740053657074656D626572004F63746F72
:104B9300626572004E6F76656D626572004465638F
:074BA300656D626572000000
:074BAA00414D00504D0000D9
:0F4BB100256120256220256520255420255900E7
:074BC000286E756C6C2900E2
:024BC7000904DF
:0E4BC900415453414D4C3231452D455642006A
:0A4BD700532F4E3A303030303100D9
:104BE100415453414D4C3231452D455642204344A9
:024BF10043007F
:104BF300415453414D4C3231452D4556422048498D
:024C030044006B
:064C0500424F4431320071
:064C0B00424F4433330068
:104C110052575720454550524F4D2070616765737B
:064C21003A2025750A008F
:104C27007475645F6364635F72785F77616E7465E0
:064C3700645F63620A00E5
:104C3D0048494420676574207265706F72743A201C
:104C4D0049443D25752C206C656E6774683D25754E
:024C5D000A004B
:104C5F0048494420736574207265706F72743A20EE
:104C6F0049443D25752C206C656E6774683D25752C
:024C7F000A0029
:104C8100415453414D4C3231452D455642204465E6
:104C91006D6F2076312E3020284A756C2020362009
:104CA100323032322C2031333A30383A3437290D10
:024CB1000A00F7
:0A4CB3005469636B2025750D0A009B
:104CBD004849442073656E64207072657373206279
:0A4CCD007574746F6E2025750A00DF
:0E4CD7002A2049525120444D4143202A0A0010
:0E4CE5002A204952512054434330202A0A000D
:0E4CF3002A204952512054434331202A0A00FE
:0E4D01002A204952512054434332202A0A00EE
:0E4D0F002A204952512054524E47202A0A00B1
:024D1D00430051
:024D1F002E0064
:104D210053756E646179004D6F6E646179005475DD
:104D31006573646179005765646E657364617900B8
:104D410054687572736461790046726964617900AF
:0A4D5100536174757264617900000B
:104D5B0005010906A101050719E029E71500250141
:104D6B0095087501810295017508810105081901E6
:104D7B0029059505750191029501750391010507AB
:104D8B0019002AFF00150026FF0095067508810003
:014D9B00C057
:054D9C00572E522E000D
:054DA1005359535400BA
:104DA60052657365742063617573653A2025730ACD
:014DB60000FC
:104DB7004E564D20706167652073697A653A2025E4
:094DC700752062797465730A001D
:104DD0005374617274206D61696E206C6F6F700A1C
:014DE00000D2
:0D4DE10055534220756E6D6F756E740A009B
:0D4DEE005553422073757370656E640A00A2
:054DFB005B25635D0073
:104E00004849442073656E642072656C6561736502
:094E100020627574746F6E0A00D3
:0D4E19002A2049525120574454202A0A00F3
:0D4E26002A2049525120525443202A0A00EC
:0D4E33002A2049525120454943202A0A00F7
:104E40002A2049525120534552434F4D30202A0ABF
:014E50000061
:104E51002A2049525120534552434F4D31202A0AAD
:014E61000050
:104E62002A2049525120534552434F4D32202A0A9B
:014E7200003F
:104E73002A2049525120534552434F4D33202A0A89
:014E8300002E
:104E84002A2049525120534552434F4D34202A0A77
:014E9400001D
:104E95002A2049525120534552434F4D35202A0A65
:014EA500000C
:0D4EA6002A2049525120544330202A0A008E
:0D4EB3002A2049525120544331202A0A0080
:0D4EC0002A2049525120544334202A0A0070
:0D4ECD002A2049525120414443202A0A0066
:0D4EDA002A2049525120444143202A0A0059
:0D4EE7002A2049525120505443202A0A002D
:0D4EF4002A2049525120414553202A0A002E
:104F010053756E004D6F6E005475650057656400F2
:0D4F11005468750046726900536174000019
:104F1E004A616E00466562004D617200417072001A
:104F2E004D6179004A756E004A756C0041756700D7
:104F3E00536570004F6374004E6F760044656300D6
:014F4E000062
:014F4F000061
:094F5000256D2F25642F25790041
:094F590025483A254D3A25530084
:0D4F620000070320041702010857104080CB
:054F6F002D494E460033
:054F74002D696E6600CE
:054F79002B494E46002B
:054F7E002B696E6600C6
:104F830009026400030100A032080B0002020200C0
:104F930000090400000102020004052400200105A9
:104FA30024010001042402020524060001070581EF
:104FB3000308001009040100020A000000070502AB
:104FC30002400000070582024000000904020001BC
:104FD3000301010509211101000122410007058395
:044FE3000340000A7D
:044FE7000009000AB3
:044FEB000008000BAF
:104FEF000A4D4355206964656E746966696361741F
:104FFF00696F6E20284453552E444944293A0A704C
:10500F00726F636573736F723A2025752C2066611A
:10501F006D696C793A2025752C20736572696573FB
:10502F003A2025752C206469653A2025752C20724D
:10503F0065766973696F6E3A2025752C2073656CE0
:0C504F00656374696F6E3A2025750A00D5
:04505B00504F520060
:04505F00455854005C
:04506300574454005A
:08506700554E4B4E4F574E0011
:0C506F0055534220726573756D650A0090
:10507B007475645F6364635F74785F636F6D706C8A
:08508B006574655F63620A00B1
:105093007475645F6364635F6C696E655F636F649B
:0850A300696E675F63620A0099
:1050AB007475645F6869645F7265706F72745F6357
:0C50BB006F6D706C6574655F63620A00C5
:1050C700427574746F6E2031205B25755D0D0A0083
:1050D700427574746F6E2032205B25755D0D0A0072
:1050E7002A204952512053595354454D202A0A002A
:0C50F7002A20495251204143202A0A007F
:105103002020202020202020206828282828202034
:10511300202020202020202020202020202020208C
:105123004810101010101010101010101010101044
:1051330084848484848484848484101010101010E4
:10514300108181818181810101010101010101013D
:1051530001010101010101010101011010101010F1
:10516300108282828282820202020202020202020E
:1051730002020202020202020202021010101020B6
:10518300303132333435363738394142434445467A
:1051930030313233343536373839616263646566AA
:0451A3004E414E002B
:0451A7006E616E00C7
:1051AC00FF510000000000204709000011520000D0
:1051BC0048090020CC51000050000000BF05000041
:1051CC00CCC74B9C4DCCC94BD74BCCE14BF34B4E86
:1051DC00018408203A100CE0FFFE1FCC1C321C325C
:1051EC00CC1C321C324C1C322008204424082028B1
:0251FC00082089
:1051FE00206861680834002200E042540139FCD571
:02520E007047E7
:1052100020686168A2680C340B78013108260025EB
:105220005B0801D20D78013105700130013A02D0DE
:08523000013EF4D1F0E77047E4
:04000003000047D5DD
:00000001FF
